:020000040000FA
:0200000079285D
:02000800CE2AFE
:1000100086110C2886150000061112203D0E1220B4
:100020001C200800BD000F308605F0303D05860419
:1000300086140000861008008316F03086048312B0
:10004000861100000615861406088610BD00861469
:1000500006088610BD1B232806118316F03086067D
:1000600083120800061100008611000086100F3070
:10007000B622303012200530B62230301220B022A5
:1000800030301220B02220301220B0222830082038
:1000900008300820013008200630082008008316A8
:1000A000F0308604831286150000061586140608B3
:1000B0008610F039BD00BD0E861406088610F03992
:1000C000BD04BD0E06118316F03086068312B022E1
:1000D0003D08080075208A110A12BC0A0319BB0AE0
:1000E000003E031908000A206A283B088A003C08E1
:1000F0008200031383129F01831606309F00803015
:1001000081003730850001308600FF3087000C14F5
:100110008312013090008515EC308F0077308E000F
:100120000B138B17B401871F3414A001A101A20186
:10013000A301AA01AF01B001B101AC01AD0186017B
:1001400032200C3008200130AE0002300820003090
:10015000BB00C730BC006A20C03008206A20C8221B
:10016000C622023008206A20C03008206A20C82237
:10017000C622023008206A20C03008206A20C82227
:10018000C622AE0BA528AF142F140B1704294C342C
:100190006F34673469346334203449344334003471
:1001A000203443346834653463346B3465347234DA
:1001B00000342034203420342034563465347234F2
:1001C0002E340034203433342E3430343034203460
:1001D0002034203400342034203462347934203404
:1001E0006D342E347934003461346D3461346D34BF
:1001F0006F3474346F34203400345B342034203452
:10020000203420345D340034AF1C1029AF1001308D
:1002100008200030BB00FD30BC006A200C300820F4
:100220002F1C16292F102C102D101E292C082D06DE
:10023000031935292C08AD002C182B2981300820F2
:100240000430AE00203084000008303E0A20840ACA
:10025000AE0B24293529B018352981300820043007
:10026000AE0020300A20AE0B3129851A50290B1719
:10027000AA08031D0429071E9221071A9E21071CA4
:10028000A421871CBB21071DCA21871DD921871ED8
:10029000E821071FFC21301C0429B01C312204294D
:1002A0000B13311C0429B11804293418592931229F
:1002B00004295B210429B201B214A701A601051D7E
:1002C000672932187A2931223214B2107A29B218E9
:1002D0007A29A70A2708093C03187029A60AA7014A
:1002E000C63008202608303E0A202708303E0A2063
:1002F0003210B214851E8029071A5F299221321507
:10030000C430082020300A2032198B294F300A20AF
:100310004B300A208F294E300A2047300A202030E7
:100320000A200800851A98292B189D292B149B292F
:100330008511C22285156430AA0008002B1CA32950
:100340002B106430AA0008002B18AC29A30A0A302D
:1003500023020318A301B1290130A3020930031CB1
:10036000A300B3210800B018AF142F14B001B101DD
:100370006430AA0008002B18C329A20A0A302202FE
:100380000318A201C8290130A2020930031CA200EF
:10039000B32108002B18D229A10A0A302102031820
:1003A000A101D7290130A1020930031CA100B3210A
:1003B00008002B18E129A00A0A3020020318A00126
:1003C000E6290130A0020930031CA000B321080077
:1003D0002B18F6292908031DFB290A30B6220C2206
:1003E0003014B010B1016430AA00FB29A001A101B2
:1003F000A201A301B3210800B01C0B2AC5300820BC
:1004000020300A2020300A208511C222851531149F
:10041000B1106430AA000800200E2104A400220EAE
:100420002304A5000B138316851083128510C222A6
:1004300024082322250823228514C222831685142A
:1004400083120B170800B5000830B600B50D03186D
:100450002B2A85102D2A85140000C222B60B262ACD
:100460000800851C3A2A341C312A311C312A851E89
:100470006F2A312A1930B622331485183310851AA1
:100480005E2AC530082020300A2020300A202F1490
:10049000331C4D2AB01470226F2AC030082002305D
:1004A000BB005830BC006A20B0010630A9006F2A9A
:1004B0004E346F346E34653421340034B114C53099
:1004C0003418C4300820331C6A2A4F300A204B30BD
:1004D0000A206F2A4E300A2047300A2032150800C1
:1004E000873008202408903C031D7E2A2508493CBB
:1004F0000319882A2508503C0319882A2008043C3F
:100500000319882A37300A20C03008203430912A55
:1005100034300A20C03008202108053C3530031D46
:1005200030300A202408453C03199B2A210803196E
:100530009B2A303E0A202208303E0A202308303E03
:100540000A2020080319AF2A043C0319AF2A863079
:1005500008202008093C2A3003192B300A20080003
:100560003C30B7000000B70BB22A0800B9000A30CF
:10057000B800BA2ABB2A0000B022B80BBB2AB90BBC
:10058000B72A08000430B62A6430B62A0530C92AD2
:100590000A30BA00C422BA0BCA2A0800F0000308C5
:1005A000F10083120C1C79280C10EC308F0077308E
:1005B0008E002A08031DAA03A80BE92AFA30A80016
:1005C0000130AC0629080319E92A2F14A90BE92ADE
:0C05D000AF1471088300F00E700E0900DB
:02400E00323F3F
:1042000043006F0070007900720069006700680069
:1042100074002000280043002900200032003000F4
:10422000310030002D003200300031003800200015
:104230006200790020004D002E00590061006D00E1
:0A42400061006D006F0074006F0054
:00000001FF
